:10000000803127290000000020008031B62309003C
:1000100000000000000000000000A80B08280800F5
:100020000130A8020001031C013EA902031C0800C4
:1000300010280130A0020001A13B031C08001E3063
:10004000A8000330A90010201928A60022008E164F
:100050000E082000A700A60E3F2022008E002000E0
:10006000452022000E082000A700A60E3F202200F7
:100070008E00200045206330A80008200800F030E2
:10008000A70526080F392704080022000E162000B5
:100090000000000000000000000000000000000060
:1000A00022000E12200000000000000000000000EE
:1000B000000000000000080022008E122000A600B0
:1000C00022000E082000A7003F2022008E00200002
:1000D00045200800A60022008E120E082000A7006E
:1000E000A60E3F2022008E002000452022000E0890
:1000F0002000A700A60E3F2022008E0020004520F1
:100100009E30A8000F30A900102008001600031927
:100110000800252086281A00800108001530A0005C
:1001200008000008A0000800A1018E2001080319A2
:100130000800860AA10AA00B9628810108008E20DB
:1001400016001A0003190800A00BA028800108005F
:100150002008031DA028800108002008031DB228E4
:1001600080010800A102031CA101210886079F2825
:1001700020080319210AA00021022008031C210ADB
:10018000FF3E86072208A000A8282108031DCA28D0
:100190008001080020081A0003190800A10BCA28D2
:1001A0008001080094202108031908008603170025
:1001B000220203190800A10BD72808009420210867
:1001C0000319E728860317001A00A10BE328800112
:1001D00008001030A800A101A001A70CA60C031C68
:1001E000F7282208A00723080318230FA107A10C52
:1001F000A00CA50CA40CA80BED2808001030A6003C
:10020000A501A401210DA40DA50D2208A402230817
:10021000031C230FA502031814292208A40723088E
:100220000318230FA5070310A00DA10DA60B02298B
:1002300008000310A00DA10DFF3E031819290800A6
:100240000310A10CA00CFF3E031820290800210078
:10025000A4012000F00101302100A00020000130A5
:100260002100A100200001302100A2002000013067
:100270002100A3002000E8010230EC00FD017D0810
:100280001F3C8031031C56296A30840020308500D1
:100290007D08AA00AB012A0884072B08853DFF30A2
:1002A0001A000130FD078031031C3F290230230072
:1002B000910015139513151413082000E300F11095
:1002C0006318F114033023009100151395131514CE
:1002D0001308FA0020000430230091001513951331
:1002E00015141308F30020000530230091001513A6
:1002F000951315141308FC0020000130EB000430A6
:10030000E4000130EE000A30E500ED01F11071105B
:10031000FA01E7019031DF222100DA01200071119A
:10032000F111F501EF01F60121000D1022000D1071
:1003300021000D108D100D118D150D168D16230039
:100340008D0121000E178E17230040309B000330D3
:100350009C009F019F1524309E0090309D0022003C
:100360000E128E1221000E128E12F0308E05200019
:100370006430A000A1018031192033305C203E3070
:10038000A8001F30A9008031102033305C20C73016
:10039000A8008031082033305C20C730A8008031AD
:1003A000082022305C20C730A80080310820283087
:1003B0006A200C306A2001306A20803140306A2087
:1003C000103025200F3025200F302520113025201A
:1003D0001E3025201E302520013025201F302520ED
:1003E00002306A20803148306A20033025200D30E9
:1003F00025200E3025200E3025200E3025200D30F2
:100400002520033025201F30252002306A2080312E
:1004100050306A200E3025200E3025200E30252049
:100420000E3025200E3025200E30252011302520BD
:100430001F30252002306A20803158306A20113068
:1004400025200E3025200E302520003025200E30AE
:1004500025200E3025200E3025201F30252002308B
:100460006A20803160306A20113025200E3025202E
:100470000F3025200F3025200F3025200E3025206D
:10048000113025201F30252002306A20803168304D
:100490006A20013025200E3025200E302520013025
:1004A00025200F3025200F3025200F3025201F302C
:1004B000252002306A20803170306A200E302520DD
:1004C0000E3025200E3025200A3025200A30252028
:1004D0000A302520153025201F30252002306A20C3
:1004E000803178306A200E302520043025200A30F3
:1004F00025200A3025200E3025200E3025200E30F4
:1005000025201F30252002306A20803101306A20EA
:100510008130210095002000303095008B168B151E
:1005200028302700940021009517911620000B1702
:100530008B176F08003C80310319BA2A50308400B1
:10054000203085006808AA00AB012A0884072B0820
:10055000853D1200E300503084002030850068089B
:10056000AA00AB012A0884072B08853D63086F07A2
:100570001A00EF017508003C8031031DC72A803145
:10058000F11DC52AE80A0F30F5008031C92AF503AC
:10059000F1118031711DD72AA43084008501DA3031
:1005A0008600870180319F209031EA247111720802
:1005B000003C80310318022BF2037208013C8031A9
:1005C000031D022BF7302100C60020000F30210050
:1005D000C7002000C0302100C8002000FF302100EB
:1005E000C9002000F7302100D60020000F30210084
:1005F000D7002000C0302100D8002000FF302100AB
:10060000D900200021002008003C8031031D0F2B61
:10061000200009302100A00020008031892B20001B
:1006200021002008013C8031031D1B2B200080315C
:10063000BA258031882B200021002008023C80311F
:10064000031D272B20008031F5258031872B2000CA
:1006500021002008033C8031031D332B2000803112
:10066000F9268031862B200021002008043C8031AF
:10067000031D3F2B20008031EB278031852B20008C
:1006800021002008053C8031031D4B2B20008831C0
:1006900097228031842B200021002008063C8031E5
:1006A000031D572B2000883136248031832B2000F6
:1006B00021002008073C8031031D632B2000883176
:1006C00085258031822B200021002008083C8031C4
:1006D000031D6F2B2000903199208031812B200049
:1006E00021002008093C8031031D7B2B2000903124
:1006F000C9218031802B200001302100A000200082
:1007000020002000200020002000200020002000E9
:10071000200020006C08013C8031031D962B220034
:100720000D1421000D1020008031AC2B6C08023C10
:100730008031031DA22B22000D1021000D1020007E
:100740008031AC2B6C08033C8031031DAC2B2200A4
:100750000D1421000D1020003E30A8001F30A9000C
:10076000803110208031992A8031B52B2008D200A9
:100770002108D3002208D4002308D5002408D6007D
:100780002508D7002608D8002708D9002808DA004D
:100790002908DB002A08DC002B08DD000408DE0045
:1007A0000508DF000608E0000708E10080310B1DA6
:1007B000982C0B116C08013C8031031D2E2C8031CC
:1007C000F11EE62B913095008031E82B1D3095000D
:1007D0008031711EF62B22008D1021008D10220019
:1007E0000D1521000D1120008031FF2B22008D14EA
:1007F00021008D1022000D1121000D1120008031EB
:10080000711E062CF60A71128031072C71167608BB
:10081000A000A1010330803123212008F7006A30B5
:100820008400203085007708AA00AB012A088407DD
:100830002B08853D1200FE007608A0000730200539
:10084000FF007E08A000A1017F088031232120083D
:10085000F700F1127718F1168031982C6C08033CE0
:100860008031031D982C6D08003C803103188F2CBB
:100870008031711C472C6D08A000A101013080312E
:100880001C212008F700770895008031632C6D0843
:10089000A000A101013080311C212008F7000230A6
:1008A00077022200A0000030031C013E003CA100A2
:1008B0002008FF3CA0002108031C013E003CA100D1
:1008C0002008200095008031F11C772C8031711CAC
:1008D000702C22008D1021008D1020008031752C8D
:1008E00022008D1421008D1020008031862C803153
:1008F000711C812C22000D1121000D11200080316E
:10090000862C22000D1521000D1120008031711C54
:100910008C2C711080318D2C71148031982C220018
:100920008D1021008D1022000D1121000D112000CD
:1009300027008031961DA72C200080310D1EA32C8E
:10094000EF038031A42CEF0A27009611200020002D
:1009500027008031961EB12C2000F1152700961239
:10096000200020008031911EE22C23001908FB009A
:1009700020007B080C3C80310318E12C7B080D3CE7
:100980008031031DD32C8A30840020308500740808
:10099000AA00AB012A0884072B08853D8001711548
:1009A000F4018031E12C8A30840020308500740805
:1009B000AA00AB012A0884072B08853D7B081A0092
:1009C000F40A91125208A0005308A1005408A20092
:1009D0005508A3005608A4005708A5005808A6000B
:1009E0005908A7005A08A8005B08A9005C08AA00DB
:1009F0005D08AB005E0884005F0885006008860023
:100A0000610887000800A0019831052221001B0819
:100A1000F8001C08F90020007808A6007908A70053
:100A20001B30A200A3018031E9202408F80025082A
:100A3000F9007808CF007908D0009831E722A43077
:100A40008400850149308600870180319F208031F4
:100A5000C0306A20803120302520203025202030F1
:100A600025207808CF007908D0009831E72222307D
:100A700084000130850049308600870180319F2045
:100A8000A430840085012230860001308700803147
:100A9000DE20A43086008701803194200430A0003D
:100AA0000230A2002230840001308500A43086008C
:100AB00087018031B820A43084008501223086006F
:100AC000013087008031DE20A4308600870180312C
:100AD000862080312E3025207808CF007908D0007C
:100AE0009831E722223084000130850049308600A9
:100AF000870180319F2022308600013087008031BD
:100B000094200330A000A4308400850122308600A8
:100B1000013087008031AD20A4308600870180310C
:100B200094200230A0000230A20022308400013064
:100B30008500A430860087018031B820A43084006D
:100B40008501223086000130870080319F20A4304B
:100B50008600870180318620803120302520563064
:100B600025204430252043302520203025202030EA
:100B7000252008006808003C8031031DF32D8031DA
:100B800080306A2080313C302520203025202030E4
:100B900025205330252070302520613025206E30EF
:100BA00025206E302520753025206E3025206730B9
:100BB00025203A30252020302520203025202030C7
:100BC00025203E3025207008003C8031031DEA2D91
:100BD00080310325F00A7008143C80310318F12D90
:100BE000F0018031F42DE80108006808003C8031F4
:100BF000031D532E803180306A2080313C30252007
:100C00002030252020302520463025206130252029
:100C1000683025207230252073302520743025203F
:100C20007530252066302520653025203A30252076
:100C300020302520203025203E3025200130230083
:100C4000910015139513151413082100A10020001D
:100C50008031C0306A20803120302520203025208E
:100C60002030252020302520210021082000CF0021
:100C7000D0019831E72249308600870180318620F3
:100C800080312030252020302520203025202030A4
:100C90002520203025202030252020302520203000
:100CA00025208031F82E6808013C8031031DED2E8F
:100CB000803180306A20803120302520203025206E
:100CC0002030252046302520613025206830252021
:100CD0007230252073302520743025207530252072
:100CE00066302520653025203A302520203025200B
:100CF00020302520203025208031C0306A2021007E
:100D00002108BF3C8031031C922E200021002108C5
:100D10007F3C80310318912E20007F302100A100FC
:100D200020002000200021002108C03C8031031851
:100D30009D2E20002100A1012000200080312030C4
:100D40002520203025203C30252020302520210062
:100D500021082000CF00D0019831E72249308600D9
:100D60008701803186208031203025203E302520AB
:100D7000203025202030252020302520203025201F
:100D800020302520203025200130EB002300910168
:100D900015139513151413082000E40002302300E6
:100DA000910015139513151413082000EE0021006F
:100DB00021082000E5009031DF22210021082000D9
:100DC000ED006D08A000A1017A08A200A301803106
:100DD000FE202008ED008031F82E01302300910024
:100DE0002100210823009300200098312122E801EE
:100DF00008006808003C8031031D562F8031803088
:100E00006A2080313C302520203025204C302520A0
:100E10006F3025206B30252061302520643025205F
:100E20007230252065302520733025207330252031
:100E3000653025203A3025202030252020302520FF
:100E40003E30252023009101151395131514130826
:100E50002100A10020008031C0306A208031203084
:100E6000252020302520203025202030252021005D
:100E700021082000CF00D0019831E72249308600B8
:100E800087018031862080312030252020302520A8
:100E900020302520203025202030252020302520FE
:100EA00020302520203025208031EA2F6808013CA1
:100EB0008031031DC22F803180306A208031203084
:100EC0002520203025204C3025206F3025206B3008
:100ED00025206130252064302520723025206530A2
:100EE00025207330252073302520653025203A30A9
:100EF000252020302520203025202030252080313D
:100F0000C0306A2021002108003C8031031D8D2F54
:100F100020007F302100A1002000200021002108B6
:100F20007F3C80310318992F200001302100A1005F
:100F300020002000803120302520203025203C302A
:100F4000252020302520210021082000CF00D001BD
:100F50009831E72249308600870180318620803130
:100F6000203025203E30252020302520203025200F
:100F7000203025202030252020302520203025201D
:100F80008031EA2F230091012100210823009300E2
:100F90002000983121220130EB002300910115132C
:100FA0009513151413082000E4000230230091006B
:100FB00015139513151413082000EE0001302300BB
:100FC000910015139513151413082000E5009031B6
:100FD000DF22E80108006808003C8831031D3A2838
:100FE000803180306A2080313C302520203025201F
:100FF0002030252046302520753025206E302520D4
:101000006B30252074302520693025206F30252055
:101010006E3025203A302520203025202030252014
:10102000203025203E3025208031C0306A2080319C
:10103000203025202030252020302520203025205C
:1010400020302520453025206E3025207430252085
:1010500065302520723025202030252020302520A5
:10106000203025202030252020302520203025202C
:101070008831962A6808013C8831031D4329803154
:1010800080306A20803120302520203025202030FB
:10109000252046302520753025206E3025206B30E8
:1010A000252074302520693025206F3025206E30B2
:1010B00025203A30252020302520203025202030C2
:1010C0002520203025208031C0306A2021002108D1
:1010D000003C8831031D7328200005302100A10049
:1010E000200088314029200021002108013C88315E
:1010F000031D9A2820008031203025202030252013
:101100003C30252020302520463025204C3025201D
:10111000203025203E30252020302520203025205D
:10112000203025202030252020302520203025206B
:1011300088313F29200021002108023C8831031D0D
:10114000C1282000803120302520203025203C304F
:101150002520203025204630252031302520203004
:1011600025203E302520203025202030252020300D
:1011700025202030252020302520203025208831B2
:101180003E29200021002108033C8831031DE82866
:101190002000803120302520203025203C302520A3
:1011A00020302520463025203230252020302520B3
:1011B0003E302520203025202030252020302520BD
:1011C00020302520203025202030252088313D2941
:1011D000200021002108043C8831031D0F29200034
:1011E000803120302520203025203C302520203023
:1011F00025204630252033302520203025203E3044
:10120000252020302520203025202030252020308A
:101210002520203025202030252088313C29200021
:1012200021002108053C8831031D3629200080312A
:1012300020302520203025203C302520203025203E
:101240004630252034302520203025203E302520F2
:10125000203025202030252020302520203025203A
:10126000203025202030252088313B2920000130E6
:101270002100A100200020002000200020002000EC
:1012800020008831962A6808023C8831031D172AFD
:101290008031C0306A2021002108013C8831031DC3
:1012A0006329200080312030252020302520203067
:1012B000252020302520463025204C302520203088
:1012C00025208831C929200021002108023C8831CD
:1012D000031D7C292000803120302520203025204E
:1012E0002030252020302520463025203130252073
:1012F000203025208831C829200021002108033C06
:101300008831031D95292000803120302520203090
:101310002520203025202030252046302520323041
:101320002520203025208831C729200021002108D0
:10133000043C8831031DAE29200080312030252057
:101340002030252020302520203025204630252023
:1013500033302520203025208831C6292000210067
:101360002108053C8831031DC5292000803120302B
:1013700025202030252020302520203025204630F3
:10138000252034302520203025202000200020007A
:101390002000200021002208003C8831031DD729AD
:1013A000200002302100A20020008831142A2000F1
:1013B00021002208013C8831031DF22920008031E0
:1013C0003C30252020302520413025205530252057
:1013D00053302520203025203E3025202030252068
:1013E0008831132A200021002208023C8831031D85
:1013F0000D2A200080313C3025202030252045302A
:101400002520493025204E302520203025203E3013
:101410002520203025208831122A2000013021008B
:10142000A20020002000200020008831962AE71723
:101430006713E71221002108013C8831031D302A7F
:10144000200021002208013C8831031D2B2A2000A6
:10145000671288312D2A20006716200088318E2AD5
:10146000200021002108023C8831031D472A20006A
:1014700021002208013C8831031D422A2000671008
:101480008831442A20006714200088318D2A2000EA
:1014900021002108033C8831031D5E2A2000210021
:1014A0002208013C8831031D592A2000E7108831A9
:1014B0005B2A2000E714200088318C2A20002100BC
:1014C0002108043C8831031D752A200021002208D0
:1014D000013C8831031D702A200067118831722A6F
:1014E00020006715200088318B2A20002100210868
:1014F000053C8831031D8A2A200021002208013C76
:101500008831031D872A2000E7118831892A2000AD
:10151000E7152000200020002000200020006708A0
:10152000E5000230EB009031DF22E8010800680896
:10153000003C8831031DE62A803180306A208031EA
:101540003C3025202030252020302520203025202B
:10155000573025206530252069302520633025202F
:1015600068302520653025206E3025203A30252032
:101570002030252020302520203025203E302520F9
:101580008031C0306A208031203025202030252055
:1015900020302520203025202030252045302520D2
:1015A0006E302520743025206530252072302520AE
:1015B00020302520203025202030252020302520D7
:1015C00020302520203025208831352C6808013C2A
:1015D0008831031D582B803180306A2080312030C3
:1015E0002520203025202030252020302520573070
:1015F000252065302520693025206330252068307E
:101600002520653025206E3025203A3025202030D9
:101610002520203025202030252020302520803115
:10162000C0306A2080313C30252020302520210028
:1016300021082000E3008831631C292B80314730CA
:101640002520723025206E3025202030252088313D
:10165000322B8031523025206F30252074302520E8
:10166000203025206308A000A10101308031232112
:101670002008E300E30A6308CF00D0019831E72295
:101680004930860087018031862080312030252036
:101690003E302520203025202030252020302520D8
:1016A0002030252020302520203025208831352C61
:1016B0006808023C8831031DE72B8031C0306A2066
:1016C000210021082000E3008831631C762B803143
:1016D000203025202030252047302520723025203D
:1016E0006E302520203025208831832B803120301A
:1016F000252020302520523025206F3025207430C1
:101700002520203025206308A000A1010130803170
:1017100023212008E300E30A6308CF00D0019831B9
:10172000E722493086008701803186202100220887
:10173000003C8831031DA32B200002302100A200B1
:1017400020008831E42B200021002208013C883150
:10175000031DC02B20008031203025203C30252067
:10176000203025204130252055302520533025209C
:10177000203025203E302520203025208831E32BC5
:10178000200021002208023C8831031DDD2B2000AF
:101790008031203025203C30252020302520453048
:1017A0002520493025204E302520203025203E3070
:1017B0002520203025208831E22B20000130210017
:1017C000A20020002000200020008831352C2100BC
:1017D00021082000E3007308003C8831031DF22B30
:1017E0008831FA2B7308013C8831031DFA2B6308FA
:1017F000083EE300E4176413E4126412E31B64166A
:10180000E411631BE4156411E31A6415E410631A10
:10181000E4146410E3196414E5176517E5166516FA
:1018200021002208013C8831031D1A2C2000E511FB
:101830008831242C200021002208023C8831031D1D
:10184000232C2000E5152000200065116319651583
:10185000E510E318E5146510631865140330EB0018
:101860009031DF227C08F200E80108006808003CA3
:101870008831031D892C803180306A2080313C30D2
:1018800025202030252020302520203025204130E3
:1018900025207530252073302520673025206130C4
:1018A00025206E302520673025203A302520203035
:1018B000252020302520203025203E302520803155
:1018C000C0306A2080312030252020302520203073
:1018D00025202030252020302520453025206E3041
:1018E00025207430252065302520723025202030B9
:1018F0002520203025202030252020302520203094
:1019000025202030252002302100A1002000883130
:10191000842D6808013C8831031D5F2D80318030A3
:101920006A208031203025202030252020302520BD
:10193000203025204130252075302520733025208A
:1019400067302520613025206E3025206730252026
:101950003A30252020302520203025202030252019
:101960002030252021002108003C8831031DBF2C98
:10197000200001302100A100200088315C2D2000D2
:1019800021002108013C8831031DF02C200080310A
:10199000C0306A208031013025208031043025207C
:1019A0008031043025208031203025202030252032
:1019B000203025204130252055302520533025204A
:1019C0002030252020302520203025205030252093
:1019D000573025204D3025202030252088315B2DA3
:1019E000200021002108023C8831031D222D200007
:1019F0008031C0306A20803144302520433025209A
:101A0000433025202030252020302520203025205F
:101A10008031033025208031023025208031003094
:101A20002520803120302520203025202030252001
:101A300050302520573025204D30252020302520BE
:101A400088315A2D200021002108033C8831031DD4
:101A5000542D20008031C0306A2080314430252050
:101A600043302520433025202030252020302520DC
:101A70002030252041302520553025205330252089
:101A800020302520203025202030252080310530B1
:101A900025208031063025208031073025208031F7
:101AA000203025208831592D200003302100A1004D
:101AB000200020002000200020008831842D2100FB
:101AC0002108013C8831031D6A2D20000130EC0003
:101AD0008831822D200021002108013C8831031D1E
:101AE000762D20000230EC008831812D200021006D
:101AF0002108023C8831031D802D20000330EC00BA
:101B0000200020002000E80108006808003C88311F
:101B1000031DD42D803180306A2080313C30252057
:101B200045302520693025206E3025207330252052
:101B300074302520653025206C3025206C30252020
:101B4000753025206E302520673025206530252012
:101B50006E3025203A3025203E3025208031C0309F
:101B60006A2080312030252020302520203025207B
:101B70002030252020302520453025206E3025209E
:101B80007430252065302520723025202030252016
:101B900020302520203025202030252020302520F1
:101BA00020302520903198286808013C8831031D99
:101BB0002B2F803180306A20803120302520453025
:101BC0002520693025206E30252073302520743083
:101BD0002520653025206C3025206C30252075307F
:101BE00025206E30252067302520653025206E3079
:101BF00025203A3025202030252021002108003CD6
:101C00008831031D0A2E200003302100A10020008E
:101C10008831282F200021002108013C8831031D34
:101C20004D2E200003302300910015139513151439
:101C300013082100A20020008031C0306A208031CA
:101C4000413025206E3025206C3025202D30252078
:101C50004B3025206F302520723025203A3025204A
:101C6000203025202030252020302520210022086A
:101C70002000CF00D0019831E7224930860087014B
:101C800080318620803120302520203025202030D2
:101C90002520203025208831272F200021002108F1
:101CA000023C8831031DDD2E20000430230091000A
:101CB00015139513151413082100A200200080317C
:101CC000C0306A2021002208003C8831031D8C2E80
:101CD00020008031573025206330252068302520B2
:101CE0002D3025204D3025206F30252064302520D3
:101CF0003A30252020302520203025205230252044
:101D00006F302520633025206F302520203025209E
:101D1000203025208831DA2E200021002208013CC5
:101D20008831031DB72E20008031573025206330C5
:101D30002520683025202D3025204D3025206F307E
:101D40002520643025203A302520203025202030E1
:101D500025202030252049302520423025202030E4
:101D6000252020302520203025208831D92E200024
:101D700080315730252063302520683025202D30D4
:101D800025204D3025206F302520643025203A3025
:101D900025202030252020302520203025202030EF
:101DA00025202030252020302520203025202030DF
:101DB0002520200020008831262F20002100210826
:101DC000033C8831031D202F2000053023009100A3
:101DD00015139513151413082100A200200080315B
:101DE000C0306A208031573025206330252068308C
:101DF00025202D302520503025206C3025207330B3
:101E000025203A3025202030252020302520203064
:101E10002520210022082000CF00D0019831E722A0
:101E2000493086008701803186208031203025208E
:101E30002030252020302520203025208831252FD6
:101E4000200001302100A1002000200020002000FF
:101E50002000903198286808023C9031031D4F28DB
:101E600021002108013C8831031D822F2000803190
:101E7000C0306A2021002208003C8831031D452F14
:101E800020007F302100A200200020002100220835
:101E90007F3C88310318512F200001302100A2001F
:101EA000200020008031413025206E3025206C300C
:101EB00025202D3025204B3025206F3025207230F5
:101EC00025203A302520203025203C302520203088
:101ED0002520210022082000CF00D0019831E722E0
:101EE00049308600870180318620803120302520CE
:101EF0003E30252020302520203025202030252070
:101F000090314C28200021002108023C8831031D1B
:101F1000F92F20008031C0306A2021002208FF3CC8
:101F20008831031D9A2F200001302100A2002000DB
:101F30008831F62F200021002208003C8831031D43
:101F4000C52F200080315730252063302520683090
:101F500025202D3025204D3025206F302520643060
:101F600025203A302520203025203C3025205230B5
:101F700025206F302520633025206F3025203E300E
:101F80002520203025208831F52F2000210022082F
:101F9000013C8831031DF02F20008031573025206F
:101FA00063302520683025202D3025204D30252018
:101FB0006F302520643025203A3025202030252020
:101FC0003C30252020302520493025204230252056
:101FD000203025203E302520203025208831F42F48
:101FE00020002100A20120002000200020009031CC
:101FF0004B28200021002108033C9031031D4A2872
:1020000020008031C0306A2021002208003C90313D
:10201000031D0F28200020302100A20020002000F6
:1020200021002208203C903103181B282000013099
:102030002100A2002000200080315730252063308D
:102040002520683025202D302520503025206C306B
:102050002520733025203A302520203025203C30A3
:10206000252020302520210022082000CF00D0018B
:102070009831E722493086008701803186208031FF
:10208000203025203E3025202030252020302520DE
:1020900020302520200020002000903198282100A9
:1020A0002108013C9031031D6628200003302300E5
:1020B0009100210022082300930020009831212262
:1020C00021002208FA0020009031962820002100EB
:1020D0002108023C9031031D7E282000043023009B
:1020E0009100210022082300930020009831212232
:1020F00021002208F30020009031952820002100C3
:102100002108033C9031031D942820000530230052
:102110009100210022082300930020009831212201
:1021200021002208FC002000200020002000E801FF
:1021300008006808003C9031031D1E298031803062
:102140006A2080313C302520203025202030252079
:10215000203025205230252069302520633025206D
:102160006830252074302520753025206E302520DC
:10217000673025203A3025202030252020302520AA
:102180003E302520023023009100151395131514BD
:1021900013082100A10020008031C0306A202100F6
:1021A0002108013C9031031DF928200080312030A6
:1021B0002520203025202030252020302520563095
:1021C00025206F3025207230252077302520613082
:1021D000252065302520723025207430252073306D
:1021E000252020302520203025202030252090312A
:1021F0001B29200080312030252020302520203050
:10220000252052302520753025206530252063306B
:1022100025206B3025207730252061302520653042
:102220002520723025207430252073302520203061
:1022300025202030252020009031C8296808013C45
:102240009031031DB629803180306A2080312030E2
:1022500025202030252020302520203025205230F8
:1022600025206930252063302520683025207430F2
:102270002520753025206E302520673025203A3006
:102280002520203025202030252020302520803199
:10229000C0306A2021002108FF3C9031031D5729DE
:1022A000200001302100A10020009031B32920003E
:1022B00021002108003C9031031D8229200080313B
:1022C0003C3025202030252020302520523025206C
:1022D0007530252065302520633025206B30252082
:1022E000773025206130252065302520723025206B
:1022F0007430252073302520203025203E302520C5
:102300009031B229200021002108013C9031031DA9
:10231000AD29200080313C30252020302520203080
:10232000252020302520563025206F302520723082
:10233000252077302520613025206530252072301A
:102340002520743025207330252020302520203092
:1023500025203E3025209031B12920002100A10107
:1023600020002000200020009031C82902302300E6
:1023700091002100210823009300200098312122A0
:10238000210021082000E300F1106318F114E80196
:1023900008006808003C9031031D182A8031803005
:1023A0006A2080313C302520203025202030252017
:1023B0002030252020302520493025206E30252052
:1023C000663025206F3025203A302520203025200A
:1023D00020302520203025202030252020302520A9
:1023E0003E3025208031C0306A20803120302520C9
:1023F0002030252020302520203025202030252089
:10240000453025206E30252074302520653025206C
:102410007230252020302520203025202030252016
:102420002030252020302520203025209031DE2A24
:102430006808013C9031031DDD2A803180306A201C
:1024400080312030252020302520203025202030CC
:10245000252020302520493025206E30252066306B
:1024600025206F3025203A302520203025202030AF
:102470002520203025202030252020302520203008
:1024800025208031C0306A2021002108003C903195
:10249000031D512A200003302100A10020009031AB
:1024A000DA2A200021002108013C9031031D7C2AFA
:1024B000200080313C302520203025202030252070
:1024C0005630252065302520723025207330252098
:1024D000693025206F3025206E30252020302520C2
:1024E000393025202030252020302520203025207F
:1024F0003E3025209031D92A200021002108023CBD
:102500009031031DA72A200080313C302520203047
:10251000252020302520763025206F3025206E3074
:10252000252020302520433025206830252072309A
:102530002520653025206730252075302520203066
:102540002520203025203E3025209031D82A20001B
:1025500021002108033C9031031DD22A2000803144
:102560003C302520203025202030252030302520EB
:10257000323025202E3025203030252031302520C6
:102580002E302520323025203030252032302520B5
:102590003030252020302520203025203E302520B9
:1025A0009031D72A200001302100A1002000200016
:1025B0002000200020009031DE2AE80108006B088E
:1025C000013C9031031DE62A9031EB2A6B08043C54
:1025D0009031031DA12B6B08013C9031031DF32AA0
:1025E000E3019031F52A1030E300E413E5136E188F
:1025F000E5176214E2146215E2156212E212621328
:10260000641B6217E213E41AE217E30A6A308400DB
:10261000203085006308AA00AB012A0884072B0834
:10262000853D62081A006210641A6214E210E4190F
:10263000E214621164196215E211E418E2156212E3
:1026400064186216E2126213E213E30A6A3084002D
:10265000203085006308AA00AB012A0884072B08F4
:10266000853D62081A006214E2146215E2156216D2
:10267000E2166213E2136E18E217E30A6A3084006E
:10268000203085006308AA00AB012A0884072B08C4
:10269000853D62081A006210651B6214E210E51A9B
:1026A000E2146211651A6215E211E519E21562126F
:1026B00065196216E212E518E216621365186217D0
:1026C000E213E30A6A308400203085006308AA0020
:1026D000AB012A0884072B08853D62081A006408AC
:1026E000A0003F302006EA006A08A0006508200626
:1026F000EA006210EA1B6214E2106A1BE214621123
:10270000EA1A6215E2116A1AE2156212EA196216F1
:10271000E2126A19E2166213EA186217E2136A18E3
:10272000E217E30A6A308400203085006308AA00BB
:10273000AB012A0884072B08853D62081A009031F6
:10274000E92C6B08023C9031031DA82B9031AD2B76
:102750006B08053C9031031D472C6B08023C9031FF
:10276000031DB62B0630E3009031B92B0630103E26
:10277000E300E4136214E2146215E2156212E2123D
:102780006213641B6217E213E41AE217E30A6A3069
:102790008400203085006308AA00AB012A08840762
:1027A0002B08853D62081A006210641A6214E21058
:1027B000E419E214621164196215E211E418E215D9
:1027C000621264186216E2126213E51B6217E213CA
:1027D000651BE217E30A6A30840020308500630835
:1027E000AA00AB012A0884072B08853D62081A005D
:1027F0006210E51A6214E210651AE2146211E5191A
:102800006215E2116519E2156212E5186216E2120C
:102810006518E21662136408A00065082006EA0045
:10282000E213EA1BE217E30A6A30840020308500D5
:102830006308AA00AB012A0884072B08853D6208BB
:102840001A0062106A1B6214E210EA1AE2146211A2
:102850006A1A6215E211EA19E21562126A19621621
:10286000E212EA18E21662136A186217E217E30A24
:102870006A308400203085006308AA00AB012A0872
:1028800084072B08853D62081A009031E92C6B08FB
:10289000033C9031031D4E2C9031532C6B08063CA9
:1028A0009031031DE92C6B08033C9031031D5C2C17
:1028B0000B30E30090315F2C0B30103EE300E41747
:1028C00064136214E2146215E2116216E2126213DA
:1028D000E41A6217E213641AE217E30A6A3084000A
:1028E000203085006308AA00AB012A0884072B0862
:1028F000853D62081A006210E4196214E21064193E
:10290000E2146211E4186215E2116418E215621211
:10291000E517E2166213651B6217E213E51AE21768
:10292000E30A6A308400203085006308AA00AB0106
:102930002A0884072B08853D62081A006210651A70
:102940006214E210E519E214621165196215E211D0
:10295000E518E215621265186216E2126408A0001A
:1029600065082006EA006213EA1B6217E2136A1B7D
:10297000E217E30A6A308400203085006308AA0069
:10298000AB012A0884072B08853D62081A006210F3
:10299000EA1A6214E2106A1AE2146211EA19621564
:1029A000E2116A19E2156212EA186216E2126A1856
:1029B000E2166217E217E30A6A30840020308500CD
:1029C0006308AA00AB012A0884072B08853D62082A
:1029D0001A000800E601E901543084002030850027
:1029E0006608AA00AB012A0884072B08853D12005F
:1029F000583C9031031DFD2CE60A543084002030F1
:102A000085006608AA00AB012A0884072B08853DCB
:102A100012004C3C9031031D882EE401E501E60ACA
:102A200054308400203085006608AA00AB012A08D3
:102A300084072B08853D1200003C90310319862E37
:102A400054308400203085006608AA00AB012A08B3
:102A500084072B08853D12002C3C9031031D342D3A
:102A6000E90AE60A9031842E6908003C9031031D82
:102A70006A2D6408A600A7010A30A200A3018031D4
:102A8000E9202408E4006608013EE200A430860044
:102A90008701803194206208A0000130A20022301A
:102AA000840001308500A430860087018031B82081
:102AB0002F3084008501223086000130870080316C
:102AC0009F20983141222D08E20064086207E4004B
:102AD0009031832E6908013C9031031DA02D6508BB
:102AE000A600A7010A30A200A3018031E920240832
:102AF000E5006608013EE200A430860087018031CF
:102B000094206208A0000130A2002230840001302D
:102B10008500A430860087018031B8202F308400E2
:102B20008501223086000130870080319F20983156
:102B300041222D08E20065086207E5009031832EEE
:102B40006908023C9031031DBE2DE7176713E71299
:102B500054308400203085006608AA00AB012A08A2
:102B600084072B08853D1200313C9031031DBB2D9D
:102B700067169031BC2D67129031832E6908033C93
:102B80009031031D0A2E54308400203085006608E1
:102B9000AA00AB012A0884072B08853D1200313CAE
:102BA0009031031DD72D0130EE009031D82DEE016C
:102BB0006508ED000430EB006408CF00D0019831C7
:102BC000E722493086008701983138223A3098311F
:102BD00031226508CF00D0019831E72249308600C4
:102BE0008701983138223A30983131226E08CF006F
:102BF000D0019831E7224930860087019831382288
:102C00000D30983131220A30983131229031DF2253
:102C10009031832E6908043C9031031D252E5430D9
:102C20008400203085006608AA00AB012A088407CA
:102C30002B08853D1200313C9031031D222E671474
:102C40009031232E67109031832E6908053C903116
:102C5000031D402E54308400203085006608AA00F1
:102C6000AB012A0884072B08853D1200313C9031C6
:102C7000031D3D2EE71490313E2EE7109031832E38
:102C80006908063C9031031D5B2E543084002030CF
:102C900085006608AA00AB012A0884072B08853D39
:102CA0001200313C9031031D582E67159031592E7A
:102CB00067119031832E6908073C9031031D832EE4
:102CC00054308400203085006608AA00AB012A0831
:102CD00084072B08853D1200313C9031031D732E73
:102CE000E7159031742EE7116708E5000530EB0019
:102CF0009031DF224F30983131226B3098313122C0
:102D00000D3098313122E60A9031102D9831042A85
:102D100054308400203085006608AA00AB012A08E0
:102D200084072B08853D1200463C9031031DD72FA8
:102D3000E401E501E60A543084002030850066088D
:102D4000AA00AB012A0884072B08853D1200003C2D
:102D500090310319D52F5430840020308500660847
:102D6000AA00AB012A0884072B08853D12002C3CE1
:102D70009031031DBF2EE90AE60A9031D32F69086E
:102D8000003C9031031DF52E6408A600A7010A300F
:102D9000A200A3018031E9202408E4006608013E76
:102DA000E200A43086008701803194206208A000F0
:102DB0000130A2002230840001308500A43086005A
:102DC00087018031B8202F308400850122308600B1
:102DD0000130870080319F20983141222D08E20088
:102DE00064086207E4009031D22F6908013C9031F9
:102DF000031D102F54308400203085006608AA007F
:102E0000AB012A0884072B08853D1200313C903124
:102E1000031D0D2F671490310E2F67109031D22FA4
:102E20006908023C9031031D2B2F54308400203060
:102E300085006608AA00AB012A0884072B08853D97
:102E40001200313C9031031D282FE7149031292FB7
:102E5000E7109031D22F6908033C9031031D462FB3
:102E600054308400203085006608AA00AB012A088F
:102E700084072B08853D1200313C9031031D432F00
:102E800067159031442F67119031D22F6908043CA7
:102E90009031031D612F5430840020308500660876
:102EA000AA00AB012A0884072B08853D1200313C9B
:102EB0009031031D5E2FE71590315F2FE7119031A0
:102EC000D22F6908053C9031031D7A2F54308400BD
:102ED000203085006608AA00AB012A0884072B0869
:102EE000853D1200313C9031031D782F9031782FB1
:102EF0009031D22F6908063C9031031D932F543036
:102F00008400203085006608AA00AB012A088407E7
:102F10002B08853D1200313C9031031D912F9031DB
:102F2000912F9031D22F6908073C9031031DAC2FAF
:102F300054308400203085006608AA00AB012A08BE
:102F400084072B08853D1200313C9031031DAA2FC8
:102F50009031AA2F9031D22F6908083C9031031D7F
:102F6000D22F54308400203085006608AA00AB01BF
:102F70002A0884072B08853D1200313C9031031D3F
:102F8000C32F9031C32F6708E5000530EB00903167
:102F9000DF224F30983131226B30983131220D30A1
:102FA00098313122E60A90319B2E9831042A543010
:102FB0008400203085006608AA00AB012A08840737
:102FC0002B08853D1200543C9831031DD628E4019E
:102FD000E501E60A54308400203085006608AA0026
:102FE000AB012A0884072B08853D1200003C98316C
:102FF0000319D42854308400203085006608AA00C4
:10300000AB012A0884072B08853D12002C3C98311F
:10301000031D0E28E90AE60A9831D2286908003C07
:103020009831031D44286408A600A7010A30A200B5
:10303000A3018031E9202408E4006608013EE20093
:10304000A43086008701803194206208A0000130FE
:10305000A2002230840001308500A4308600870160
:103060008031B8202F308400850122308600013065
:10307000870080319F20983141222D08E2006408AA
:103080006207E4009831D1286908013C9831031D9A
:10309000712854308400203085006608AA00AB01F6
:1030A0002A0884072B08853D1200313C9831031D06
:1030B0005B2898316B2854308400203085006608E6
:1030C000AA00AB012A0884072B08853D1200673C43
:1030D0009831031D6E28651498316F28651098315A
:1030E000D1286908023C9831031DD128543084004E
:1030F000203085006608AA00AB012A0884072B0847
:10310000853D1200313C9831031D8928E515983121
:103110008A28E5117308003C9831031D9228E403C6
:1031200098319C287308013C9831031D9C28640841
:10313000033EE40098319C286408A600A7010230F1
:10314000A200A3018031E9202408E300E4176413FE
:10315000E4126412E31B6416E411631BE4156411AA
:10316000E31A6415E410631AE4146410E319641498
:10317000E5176517E5166516651163196515E51000
:10318000E318E5140630EB009031DF224F30983120
:1031900031226B30983131220D30983131227C0848
:1031A000F200E60A9031EA2F9831042A5430840064
:1031B000203085006608AA00AB012A0884072B0886
:1031C000853D1200533C9831031D13295430A20051
:1031D000A430860087018031D22021082200B80067
:1031E0003808003C98310318102920000230EC0008
:1031F0005030983131227730983131227230983105
:1032000031222030983131226F30983131226630AE
:10321000983131226630983131220D309831312287
:1032200020009831042A543084002030850066083C
:10323000AA00AB012A0884072B08853D1200473CF1
:103240009831031D4D294F30A200A430860087011C
:103250008031D22021082200B8003808003C983183
:1032600003184A2920000130EC00503098313122F7
:1032700077309831312272309831312220309831B4
:1032800031226F30983131226E30983131220D3039
:103290009831312220009831042A543084002030A3
:1032A00085006608AA00AB012A0884072B08853D23
:1032B0001200593C9831031DC5295930A200A43091
:1032C000860087018031D22021082200B80038080A
:1032D000003C98310318C22920006C08013C983149
:1032E000031D8929503098313122773098313122AD
:1032F0007230983131222030983131226F3098313C
:1033000031226E30983131220D309831312298318E
:10331000C2296C08023C9831031DA829503098310D
:103320003122773098313122723098313122203079
:10333000983131226F309831312266309831312204
:103340006630983131220D30983131229831C229BE
:103350006C08033C9831031DC22941309831312259
:103360006E30983131226130983131226C30983191
:1033700031226F30983131226730983131220D304F
:103380009831312220009831042A543084002030B2
:1033900085006608AA00AB012A0884072B08853D32
:1033A0001200563C9831031D042A5630A200A43066
:1033B000860087018031D22021082200B800380819
:1033C000003C98310318032A2000563098313122EE
:1033D0006530983131227230983131227330983112
:1033E00031226930983131226F30983131226E307C
:1033F00098313122203098313122393098313122C0
:103400000D30983131222000080021009E178F30A6
:103410009E0530309E042000A00DA00D7C302005BC
:1034200021009D001D1420001330A80080310820C9
:1034300021009D149D18FE331D102000111308005B
:103440000800230015139513151555309600AA3062
:10345000960095149518FE331511200012120800DD
:103460000800111A0132FD3323009A0020000800E1
:1034700016000319080098313122FA3308009831F8
:10348000402AAD01AE012F308600870180319420A3
:1034900021082200B8003808053C98310318522A48
:1034A0002000080020002F30860087018031942002
:1034B00021082200B8003808053CB8002000303050
:1034C000A000220038082000A10022308400013032
:1034D00085008031C52039308400013085002230DC
:1034E00086000130870080319F2020089831031921
:1034F0007F2A84032F30860087018031A0202F305F
:1035000084008501393086000130870080319F209A
:103510000630C5000130C700C8019831A522983196
:103520009822983198229831982298319822080050
:103530004708A6004808A7000A30A200A30180316E
:10354000E9202408C7002508C800C5032F308600DD
:103550008701803194204508A0000130A20022306C
:103560008400013085002F30860087018031B8202B
:103570002230840001308500803191202008C6006F
:1035800030304602C6004608A600A7014708A20040
:103590004808A3008031E92024082200A000200070
:1035A00025082200A10020002D0822002007A000ED
:1035B00020002E080318013E22002107A100200848
:1035C0002000AD00220021082000AE000800850187
:1035D0004930840051104F08A4005008A500103055
:1035E000A2002730A30098310A23E830A20003305C
:1035F000A30098310A236430A200A30198310A2362
:103600000A30A200A30198310A2324089831182314
:10361000800108002408A0002508A1008031FE20B8
:10362000200898310319152B51149831511C1B2B6C
:08363000303E8000013108006A
:020000040001F9
:04000E00C20FFF1D01
:00000001FF
